:020000002729AE
:10000800080064001B20031805286920A80108308F
:10001800A3006A201B200318A80AAB1EA801A20C83
:10002800A30B0D28AB1AA2136A20220808003A086D
:100038008400380884178004841300052B1B3806B5
:10004800FF3E0800A4002908031922291D21A00049
:100058002518831724088400200880008313A40A25
:10006800A9032728A6003A088400F030B70508300D
:10007800A70003100318B70A4F20A60CA70B3E28A9
:100088000000AB1A370C4F20252103144F202F08EE
:10009800A3002E0896288413AB1F5E280008380496
:1000A8002B1F38068000841700083804031C380604
:1000B80080006A2800083804031C38062B1B380601
:1000C80080008417380980056A2837172B081F39DC
:1000D800003EA1002A080E3E0318A10A371FA328D4
:1000E8003713A0000230C720A32800308A00280850
:1000F80007398207013402340434083410342034B8
:100108004034803483178001840AFF3E031D87280A
:10011800222903178D0083168C130C1483120C08E4
:100128002229A301A200FF30A207031CA307031C76
:1001380022290330A100E730A3209728A101FC3E23
:10014800A000A109031CAE28FF300000A007031877
:10015800A928A0076400A10FA8280800A8007920F2
:10016800A001A101A81DA000A819A100200822290A
:100178000310A00DA10DFF3E0318BC28200822295A
:100188000310A10CA00CFF3E0318C4282008222944
:10019800A101A301A2000230DB28A101A301A20052
:1001A8000130DB28A101A301A2000430DB28A8004C
:1001B80023082102031DE228220820020430031824
:1001C8000130031902302805031DFF3022291030A1
:1001D800A600A501A401210DA40DA50D2208A402C5
:1001E8002308031C230FA502031801292208A407CA
:1001F80023080318230FA5070310A00DA10DA60BB4
:10020800EF28200822291030A800A101A001A70C7E
:10021800A60C031C15292208A00723080318230F7E
:10022800A107A10CA00CA50CA40CA80B0B29240851
:100238002229840031088A003008820083130313BE
:100248008312640008002030840060308A0187200F
:10025800A030840050308A0187201030840060303C
:100268008A0186209030840060308A0186208316B7
:1002780007309F0099018312980183160230980075
:100288008312EF01F001831686100611880107100A
:100298008710071187128312D2010130A300F430AE
:1002A8008A01962087120A308A0195208716013024
:1002B800A300F4308A0196208A110A12942E07149A
:1002C8000A308A01A220071008008A110A12A42203
:1002D8006808A000A1010830A200A3018A01EB2050
:1002E800DC006808A000A1010830A200A3018A016F
:1002F800EB202408B2002508B30032088A01B22096
:10030800E7008710B8305C0788008A016321403015
:10031800620788008A0163218A110A126F22640029
:100328005E08003C8A110A12031DA0295B086704B5
:1003380088008A110A12A3295B08670688008A01C7
:100348006321080087103E3088008A0163218614E3
:1003580006110130D3006400033053028A110A12D7
:100368000318F129B830D6006400C03056028A114B
:100378000A120318E12987108A0163214030880096
:100388008A016321560888008A0163218714013095
:10039800D7006400413057028A110A120318DC2979
:1003A80088018A016321D70A8A110A12031DCD29FF
:1003B800D60A8A110A12031DB829831086188314D5
:1003C80006198614061D861083180615831C061147
:1003D800D30A8A110A12031DAF2987108614061141
:1003E8000130D3006400033053028A110A12031843
:1003F800212A3E3088008A016321C03088008A01A2
:100408006321403088008A016321B83088008A015E
:1004180063213F3088008A01632183108618831482
:1004280006198614061D861083180615831C0611E6
:10043800D30A8A110A12031DF62986140611871495
:1004480008006008D3006400530861028A110A1288
:10045800031C3D2A5308E3006508E8008A01692166
:100468006608E8008A016921D30A8A110A12031D65
:10047800272A6508D3006400530866028A110A1205
:10048800031C552A5308E8006008E3008A01692123
:100498006108E3008A016921D30A8A110A12031D3F
:1004A8003F2A08008A110A12A4226808A000A101A4
:1004B8000830A200A3018A01EB20DC00871040303D
:1004C800620788008A016321B8305C0788008A01C6
:1004D8006321871408008A110A12A422871483163C
:1004E800FF3088008312071507140A308A01A220FA
:1004F8000808DB0007100A308A01A22007140A3016
:100508008A01A2200808DB0007100711831688015A
:10051800831287104030620788008A016321B8304F
:100528005C0788008A016321871408008A01562223
:100538008A016F225B08510488008A016321080040
:100548006400403063028A110A12031CB32A861021
:10055800061540306302E2008A110A12B72A86148F
:1005680006116308E20008000130DE008A016921F3
:10057800DE01080088018A016321E30A8A01562204
:100588000800640063083F3C8A110A12031DED2A23
:10059800871083108618831406198614061D861082
:1005A80083180615831C0611403088008A016321D0
:1005B8006808A000A1010830A200A3018A01EB206D
:1005C800B2002108B300B830320788008A016321DD
:1005D800871408005F084F07E30064085007E80025
:1005E8008A0169215F084F02E30064085007E800A8
:1005F8008A0169214F085F07E30064085002E80098
:100608008A0169215F084F02E30064085002E8008C
:100618008A01692164084F07E3005F085007E80072
:100628008A01692164084F02E30050085F07E80067
:100638008A0169214F086407E3005F085002E80057
:100648008A01692164084F02E3005F085002E8004C
:100658008A01692108008714D0304E07B200FF30A4
:100668000318013EB3003208A6003308A700033080
:10067800A200A3018A010721B2002508B3000030B7
:100688003207C80002304807C9004808C70064009C
:10069800470849028A110A12031C5E2B47088A017F
:1006A8008D2088008A016321E30AC70A8A110A1289
:1006B800031D4B2B8A0156228A01BE2208006C08B2
:1006C800E3006E08E800640068086D028A110A12E7
:1006D800031C752B8A016921E80A8A110A12031D75
:1006E800672B6C0AE3006E08E800640068086D0276
:1006F8008A110A12031C882B8A0169216A08E807F3
:100708008A110A12031C792B08006E08E8006C088D
:10071800E300640063086B028A110A12031C9B2B16
:100728008A016921E30A8A110A12031D8D2B6E03BF
:10073800E8006C08E300640063086B028A110A127F
:10074800031CAE2B8A0169216A08E3078A110A1281
:10075800031C9F2B080060086102D8006508660228
:10076800DA00C501C6016508E8006008E300640016
:10077800630861028A110A12031CDD2B5A08C50797
:100788000318C60A4508A0004608A10058088A01AF
:10079800D7208A110A12031DD62B5A08C502031C3A
:1007A800C603E80A8A016921E30A8A110A12031DAD
:1007B800BB2B0800DF015D08E40003105D0DB200EB
:1007C800B301B30D3208033CC5003308031C013ED6
:1007D800003CC60064005F0864028A110A12031C08
:1007E800342C8A01EE2264008A110A12C61F142CC6
:1007F8000430A600A7015F08A200A3018A0107210F
:10080800B2002508B3000630B2070318B30A32084D
:10081800C50733080318013EC6078A110A12312C8E
:1008280064085F02B200B301031CB3030430A600DE
:10083800A7013208A2003308A3008A010721B200E9
:100848002508B3000A30B2070318B30A3208C507EF
:1008580033080318013EC607E403DF0A8A01EE2BBA
:10086800080053083C3E84000008B200FF30A20094
:10087800A20A22080F3C8A110A12031C642C8A114E
:100888000A12502432028A110A12031D3C2C220833
:10089800E9008A110A12642C04308A0022088207AF
:1008A8003034313432343334343435343634373404
:1008B80038343934613462346334643465346634CA
:1008C8000800DF015D08E40003105D0DB200B3010C
:1008D800B30D3208033CC5003308031C013E003C3D
:1008E800C60064005F0864028A110A12031C9E2C69
:1008F8008A01EE2264085F02B200B301031CB3034D
:100908000430A600A7013208A2003308A3008A0118
:100918000721B2002508B3000A30B2070318B30A4A
:100928003208C50733080318013EC607E403DF0A87
:100938008A01752C0800DF015D08E40003105D0DD5
:10094800B200B301B30D3208033CC5003308031CE1
:10095800013E003CC60064005F0864028A110A1266
:10096800031CD02C8A01EE220430A600A7015F08E0
:10097800A200A3018A010721B2002508B3000630AE
:10098800B2070318B30A3208C50733080318013E33
:10099800C607DF0A8A01AF2C0800DF015D08E40002
:1009A80003105D0DB200B301B30D3208033CC5005E
:1009B8003308031C013E003CC60064005F08640263
:1009C8008A110A12031C0B2D8A01EE2264085F02A9
:1009D800B200B301031CB3030430A600A701320818
:1009E800A2003308A3008A010721B2002508B3003A
:1009F8000A30B2070318B30A3208C50733080318C8
:100A0800013EC6070330E402DF0A8A01E12C080030
:100A1800510888008A016321E30A64006308403CA6
:100A28008A110A12031D292D8610061587104030D9
:100A380088008A016321C03088008A016321B830A8
:100A4800590788008A016321871464006308803C81
:100A58008A110A12031D4B2DD90A64005908083C53
:100A68008A110A12031D392DD901E30186140611D2
:100A78008710403088008A016321B8305907880000
:100A88008A016321C03088008A0163218714080025
:100A98006008D3006400530861028A110A12031C1B
:100AA800702D6508D6006400560866028A110A127D
:100AB800031C6A2D5308E3005608E8008A016921DF
:100AC8006A08D6078A110A12031C572D6A08D30729
:100AD8008A110A12031C4E2D08000730BA00803014
:100AE800B8002030AA00AB018A0105205D3C8A11BC
:100AF8000A12031D782D0430A9000530B000B10199
:100B0800A5013C308A012620D30164000430530239
:100B18008A110A1203189C2D8A01352453083C3E79
:100B2800840069088000D30A8A110A12031D892DDE
:100B38003C08A000A10104308A01BF20B2002108AE
:100B4800B3003D083204CA003E08A000A1010430E9
:100B58008A01BF20B2002108B3003F083204CB004D
:100B680008000730BA008030B8002030AA00AB0176
:100B78008A0105205D3C8A110A12031DBC2D06302E
:100B8800A9000530B000B101A5013C308A0126203A
:100B9800D3016400063053028A110A120318E02DAB
:100BA8008A01352453083C3E840069088000D30A32
:100BB8008A110A12031DCD2D3C08A000A1010430A2
:100BC8008A01BF20B2002108B3003D083204CA00E0
:100BD8003E08A000A10104308A01BF20B20021080C
:100BE800B3003F083204CB004008A000A101043044
:100BF8008A01BF20B2002108B30041083204CC00AA
:100C080008000730BA008030B8002030AA00AB01D5
:100C18008A0105205D3C8A110A12031D0C2E8A01E7
:100C28000520E90030306902EA006A08A0000130B6
:100C38008A01D620B2006A08A00009308A01D120B2
:100C4800B400320834048A110A12031D052E080064
:100C58000730BA008030B8002030AA00AB018A0102
:100C680005205D3C8A110A12031D332E0830A900A5
:100C78000530B000B101A5013C308A012620D3011E
:100C88006400083053028A110A120318572E8A0189
:100C9800352453083C3E840069088000D30A8A1131
:100CA8000A12031D442E3C08A000A10104308A0149
:100CB800BF20B2002108B3003D083204E0003E081E
:100CC800A000A10104308A01BF20B2002108B300AE
:100CD8003F083204E1004008A000A10104308A0165
:100CE800BF20B2002108B30041083204E5004208E1
:100CF800A000A10104308A01BF20B2002108B3007E
:100D080043083204E60008004A08CF004B08D00028
:100D18004C08DD0008004A08E3004B08E80008001A
:100D28008A01A6210830E3003F30E8008A015622F4
:100D3800D3016400173053028A110A120318EF2EE8
:100D48005308163C8A110A12031CCC2E8A110A1267
:100D5800B126CE008A110A12CC2E06308A0053081A
:100D68008207473452344134503448344934433488
:100D78002034443445344D344F34203442345934CB
:100D8800203443344F344D3450345334593453346D
:100D980064004E08203C8A110A12031DE62E013019
:100DA800D6006400033056028A110A120318E32E93
:100DB8008A01BE22D60A8A110A12031DD52E8A116B
:100DC8000A12E82E8A012F238A01BE22D30A8A1129
:100DD8000A12031D9D2E4030CF002030D00016305F
:100DE800DD008A01DE238A019F248A0165240530FB
:100DF800DD008A01DE238A019F240230DD008A019A
:100E0800DE230130DD008A01DE23E0017F30E100CE
:100E1800E5013F30E6008A0125220230E0007D30FE
:100E2800E1000230E5003D30E6008A012522073066
:100E3800BA004030B8002030AA00AB01AE01AF01C3
:100E480052308A01362065308A01362061308A01A5
:100E5800362064308A01362079308A0136203A30CB
:100E68008A0136200A308A0136200D308A01362060
:100E78000730BA008030B8002030AA00AB018A01E0
:100E880005205D3C8A110A12031D432F8A010520A3
:100E9800E9006908A00063308A01CC20B200690823
:100EA800A00043308A01CC20B400320834048A15EB
:100EB8000A12031D81286908A00073308A01CC201A
:100EC800B2006908A00053308A01CC20B40032086F
:100ED80034048A150A12031D89286908A000713094
:100EE8008A01CC20B2006908A00051308A01CC20C8
:100EF800B400320834048A150A12031D91286908BF
:100F0800A00074308A01CC20B2006908A0005430D7
:100F18008A01CC20B400320834048A150A12031D51
:100F280099286908A0006C308A01CC20B2006908B1
:100F3800A0004C308A01CC20B400320834048A1551
:100F48000A12031DBB286908A00072308A01CC2050
:100F5800B2006908A00052308A01CC20B4003208DF
:100F680034048A150A12031DA9286908A0006230F2
:100F78008A01CC20B2006908A00042308A01CC2046
:100F8800B400320834048A150A12031DA12869081E
:100F9800A0006B308A01CC20B2006908A0004B3059
:100FA8008A01CC20B400320834048A150A12031DC1
:100FB800CC286908A00064308A01CC20B2006908F6
:100FC800A00044308A01CC20B400320834048A15C9
:100FD8000A12031DC3286908A00065308A01CC20C5
:100FE800B2006908A00045308A01CC20B40032085C
:100FF80034048A150A12031DC1286908A00070303C
:101008008A01CC20B2006908A00050308A01CC20A7
:10101800B400320834048A150A12031DD02869085E
:10102800A00075308A01CC20B2006908A0005530B4
:101038008A01CC20B400320834048A150A12031D30
:101048007E296908A00078308A01CC20B20069089E
:10105800A00058308A01CC20B400320834048A1524
:101068000A12031D88296908A00079308A01CC205A
:10107800B2006908A00059308A01CC20B4003208B7
:1010880034048A150A12031D96296908A0006630DF
:101098008A01CC20B2006908A00046308A01CC2021
:1010A800B400320834048A150A12031DAF286908EF
:1010B800A00068308A01CC20B2006908A00048303E
:1010C8008A01CC20B400320834048A150A12031DA0
:1010D800EB286908A00076308A01CC20B2006908A4
:1010E800A00056308A01CC20B400320834048A1596
:1010F8000A12031D35298A011B2F8A01B5258A0189
:1011080088268A01DE238A011B2F8A01B5258A01D8
:1011180088268A019F248A011B2F8A01B5258A0106
:1011280088268A0165248A011B2F8A01B5258A0130
:1011380088268A01D1248A011B2F8A012C268A013C
:1011480005268A014C258A011B2F8A012C268A0133
:1011580025228A011B2F8A010526E0017F30E10044
:10116800E5013F30E6008A014C258A011B2F8A01E0
:101178002C268A01AF238A011B2F0130DE008A0149
:1011880071258A018F268A016921DE018A011B2FB8
:101198008A01A6218A011B2F8A0171258A018F26BF
:1011A8000730BA008030B8002030AA00AB018A01AD
:1011B80005205D3C8A150A12031DDB288A010520DB
:1011C800CE008A0156228A012F238A011B2F8A0109
:1011D80071258A018F268A0156226308EF0007309D
:1011E800BA008030B8002030AA00AB018A0105207F
:1011F8005D3C8A150A12031DFA288A010520CE00D3
:1012080064004E08403C8A150A12031933298A01E2
:101218002F236400803063028A150A12031C1629E2
:101228006F08E30064004E083B3C8A150A12031954
:101238001F298A01BE220730BA008030B80020304A
:10124800AA00AB018A0105205D3C8A150A12031D1C
:1012580026298A010520CE008A150A1204298A0146
:101268001B2F8A0171258A018F266308EF00680801
:10127800F0008A0156220730BA008030B8002030CA
:10128800AA00AB018A0105205D3C8A150A12031DDC
:1012980046298A010520CE0064004E08403C8A1584
:1012A8000A1203197C298A012F236F08E3000830EA
:1012B800E8076400403068028A150A12031C662990
:1012C8007008E8008A0156220730BA008030B8005A
:1012D8002030AA00AB018A0105205D3C8A150A125C
:1012E800031D6F298A010520CE008A150A1250298C
:1012F8008A011B2F8A01B5258A018F264C08D10047
:101308008A019A228A011B2F8A01B5254A08EC0016
:101318004B08EB004C08EE008A0105268A01892358
:101328008A011B2F8A01B5254A08EE004B08ED00FB
:101338004C08EC008A0105268A0163238A011B2FC9
:0813480063008A150A12A429B2
:02400E00753DFE
:00000001FF
